:030000000219FDE5
:03000B000200A848
:03002B0002019738
:03005B000203415C
:030073000203275E
:1000800002030406080C10182030406080040608A3
:100090000C10182030406080A0C000070F1F3F05E3
:1000A000050D050305030302C2AF306308C2638573
:1000B0007C8AD2AF32C0D0C0E0206227E525600242
:1000C000E473E525F4C3334009758A00D263F57CF7
:1000D00001D4F58A758B00758D00D262D0E0D0D046
:1000E000D2AF32C3E526334009758A00D263F57C6E
:1000F00001F4F58AC262E526F4603B3068032072A1
:1001000013758B00758D00D0E0D0D0C292C294C21E
:1001100096D2AF32C292C294C296206E0C2066096B
:10012000740AD5E0FDE57E4290758B00758D00D098
:10013000E0D0D0D2AF32758A00D263757C00C28D18
:10014000D262212901C2306805206602D29201C222
:10015000306805206602D29401C23068052066022C
:10016000D29601C2C29330680A2066077408D5E0AF
:10017000FDD29201C2C29530680A2066077408D584
:10018000E0FDD29401C2C29730680A206607740865
:10019000D5E0FDD29601C2C2AFC2AD53E6EFC0D0EA
:1001A000C0E0D2D3D2AFE57D6009E57A6005757A0B
:1001B0000041D4757A01C2CEE52A60072074491542
:1001C0002A41087800790020742EE580307E01F401
:1001D00030E60278FF53DACF207E0343DA20307E08
:1001E0000343DA10C2D8C271E580307E01F430E6F4
:1001F0000279FFC3E89970CB306103752A18207427
:1002000003752A18885FD27020740DE52B600415E1
:100210002B411843DA01C2D8207002417AA85F202E
:100220006102C270207431C3E894F0400374F0F8A6
:10023000E8C4540F28F87984B703024158C313C3A4
:10024000138721200802C313200A06C3C898F84167
:100250005828F8500374FFF8C3E895685003E56820
:10026000F88822E52D54066011E533C313C3132427
:10027000062522F52250037522FF852224A824C3D7
:10028000E52495644002A8648825E569700241BEB2
:10029000C3E8AA699A5003E8FAE4F9EAC333FBE534
:1002A0006BF45B29400D256AF8E56A6002156A4027
:1002B0000B41BE0AC3E56A9A5002056A78FF882698
:1002C000C26EC3E52694F84002D26EC3E525944081
:1002D0004002D26420CF0AD0E0D0D043E610D2ADA5
:1002E00032C2CF053AE57D6009E57B6005757B008C
:1002F000611D757B017801E52A6005307402152ABD
:10030000C3E55F94014005756200611D756300756A
:100310006C00E5622401F56250037562FFD0E0D005
:10032000D043E610D2AD32C2AFC0D053E67FC26038
:10033000759100855694855795759104D0D0D2AFAC
:1003400032C2AF53E6EFC2ADC0D0C0E0C0F0D2D3EE
:10035000D2AFA8FBA9FCE57D6007C3E913F9E81358
:10036000F8C2D830710261B353DACF207E0343DA8A
:1003700010307E0343DA20D271E580307E01F42014
:10038000E602618A88278928A1DA53DACF207E0322
:1003900043DA20307E0343DA10C2D8C271307402CF
:1003A000A1C67800E580307E01F430E602A1C6885F
:1003B0005FA1AE53DACF207E0343DA20307E0343C1
:1003C000DA10C271206102818C53DACF207E0343A0
:1003D000DA10307E0343DA20C2D8D271885A895BA2
:1003E000C3E89558F8E99559F97B007E087A00C36F
:1003F000E8948CE994005005755E00817E88217830
:10040000A2E6A8216055C3E894C8E994005008E426
:10041000D2E4FB7A0A8159C3E89468E99401500850
:10042000E4D2E3FB7A0F8159C3E894D0E9940250F7
:1004300008E4D2E2FB7A1E8159C3E894A0E994054E
:100440005008E4D2E1FB7A3C8159C3E89498E994DE
:10045000085008E4D2E0FB7A787E00C3E8955CFCA3
:10046000E9955DFD30E70AECF42401FCEDF434007D
:0E047000FD755E00C3EC9AED9E5003755E01B3
:10047E00885C895D855A58855B597802A1AEC3E8C0
:10048E009527F8E99528F9307C02A192307B02A1DC
:10049E0092307A02A18B20750281AFE9FDE8FC81D2
:1004AE00CEE9C313F9E813F8307902A18BE9C3132F
:1004BE00F9E813F8307802A18BE9C313FDE813FCB9
:1004CE00206126C3EC941CED9402400281E5ED7090
:1004DE0018C3EC94C850120529C3E529940A50029A
:1004EE00A1C6755F00D270A1C6E5296002152978F4
:1004FE0088E6F97400207F087896B90302789EE6A4
:10050E0024FAFEE43400FFC3EC9EFCED9FFD92083E
:10051E00B90310A2085007207609D276A1313076A1
:10052E0002C276A2085016B9030DECF42401FCEDBC
:10053E00F43400FD02054B78007900A192B9031541
:10054E00EC33FCED33FDC3EC940AFCED9400FD504E
:10055E00047C007D00C3EC94FFED9400400678FF10
:10056E007900A192EC8575F0A4C5F0A2F733F87965
:10057E000040030205AE78FF79000205AEE9C31311
:10058E00F9E813F8307C0EE9600278FFC3E81338FF
:10059E00F8E43400F9C3E894FFE99400400278FFD0
:1005AE00885FD270206102A1C6741FF4552F4BF5DF
:1005BE002FC274EB7002D274752A18307403752A28
:1005CE000A306102A1DA20740353DAFE2074037537
:1005DE002B06D0F0D0E0D0D0D2AD43E61032790168
:1005EE0002060A790302060A790A02060A791E022F
:1005FE00060A796402060A79C802060A7817E4D553
:10060E00E0FDD8FAD9F6227A147B780206317A10F8
:10061E007B8C0206317A0D7BB40206317A0B7BC8D5
:10062E000206317902B27DE4C295D5E0FDD294D5B1
:10063E00E0FDC294D5E0FDD295D5E0FDD292E576EF
:10064E00D5E0FDC2927496D5E0FDD9D9EAF8D5E091
:10065E00FDD8FBDBCEC29522C37C007D0075F00079
:10066E0005F0EA33FAEB33FB50F6EB13FBEA13FA21
:10067E00C3E9FFE8FEE89AF8E99BF95004EFF9EEBA
:10068E00F8B3EC33FCED33FDD5F0DFEDF9ECF822E9
:10069E00E889F08A20D2D4F8A9F07B0030F70B7BE2
:1006AE00FFF42401F8E9F43400F9E88520F0A4AD54
:1006BE00F0F8E98520F0A4AFF0FEED2EF974003FBE
:1006CE00FA7C04C3EA13FAE913F9E813F8DCF48BA5
:1006DE00F030F70AE8F42401F8E9F43400F9E88977
:1006EE00F0C2D4F8A9F02222C3E54113F9E5401374
:1006FE00F8C3E54598F8E54699F9500CC3E894809F
:10070E00E994FF401602072DC3E8947FE994005048
:10071E000302072D787F790002072D788079FF88F4
:10072E004A894B22E54A2547F8E54B3548F9854B72
:10073E0020E4300701F43549FA30E709C3EA94F0B2
:10074E00401502076BC3EA940F500302076B78FF44
:10075E0079FF7A0F02076B780079007AF0C3E524EF
:10076E009564500AC374019524500B020789E54B1A
:10077E0020E70E020789E54B30E706884789488A4D
:10078E00492278A4E6FAC3E54A33F8E54B33F9D1AA
:10079E009EE930E70BC3E89480E994FF4013E1C370
:1007AE00C3E8947FE994005002E1C3787F7900E1B9
:1007BE00C3788079FFE820E715C3E52398F8400950
:1007CE00C3E8940140030207EA78010207EAE8F45D
:1007DE0024012523F840030207EA78FF884C22788B
:1007EE00A5E6FAA848A949D19EE930E70CC3E894DA
:1007FE0001E994FF401602081EC3E894FFE9940035
:10080E00500302081E78FF790002081E780179FF56
:10081E00E920E715C3E54C98F84009C3E894014078
:10082E00030208457801020845E8F42401254CF836
:10083E00400302084578FF88242278FFC2642069AD
:10084E003D206A12D264C3E541940A4009C3E525EE
:10085E0094405002C26479A1E76023E541601F74A1
:0F086E00FF8541F0848539F0306A0375F005A4E9
:10087D00F8C5F0600278FFC3E895675002A8678855
:10088D006622C3E54094C8E5419400E56650031423
:10089D0001A0046002F566220208A82275E89022E4
:1008AD007883E6FFE5E820ECF7A8BDA9BE0573C384
:1008BD00E57394084052757300E9FA79A0E7604436
:1008CD00EA7007E574601B0208E3C3E895746010D5
:1008DD00E5745006600C140208EF0460F90208EF8D
:1008ED00E574F574C39472401B7564C0C3940440E1
:1008FD0013756480C39404400B756440C394044025
:10090D000375640075BB0922E564F460020564E5B6
:10091D0073B4070375BB1022743279A687F0A4C592
:10092D00F0A2F733F8C3E895644002A864882288E2
:10093D0024882588268867227540007541F022C2DB
:10094D00AF75C820A8CCA9CDAA3A30CF010A75C879
:10095D0024D2AFC3EA13FAE913F9E813F8AB3BACB1
:10096D003C883B893CC3E89BF8E99C20690A547F8D
:10097D00F9306702416F21CCAD3D8A3DF9EA9D54B6
:10098D007FFA600478FF79FFAE3EAF3F8B3E8C3F20
:10099D00C3EC9FFCC3E99CF542A83BA93CC3E89E70
:1009AD00F8E99FF9C3E54113FBE54013FAE82AF591
:1009BD0040E93BF54150067540FF7541FF4116AAD0
:1009CD0040AB41AC40AD417E047F02C3EB9404408B
:1009DD00021E1FC3EB940840021E1FC3ED13FDEC56
:1009ED0013FCDEF7C3EA9CFAEB9DFBEF6009C3E94C
:1009FD0013F9E813F8DFF7EA28FAEB39FB8A408B95
:100A0D004150067BFF8B408B41C3EB94025002D2C9
:100A1D00673069047F0341417892E6FFC3E537945F
:100A2D008240110FC3E53794A040010FC3EF940628
:100A3D0040027F057E02E541C4540FF9E541C454DF
:100A4D00F0F8E540C4540F28F8C3E89EFAE9940085
:100A5D00FB4009C3EA9402EB940050047A02E4FBD4
:100A6D0041BBAA40AB41EBC4FEEAC4540F4EFCC3DC
:100A7D00EA9CFAEB9400FBC3E813C313F8EA28FAD7
:100A8D00EB3400FB8A408B41C3EB94024002C267FA
:100A9D007802EBC4FE7B00EAC4540F4EFAC3EA9809
:100AAD00FA4005C3940250027A027892E6FF306054
:100ABD000241BB855256855357D26043E680C3E44D
:100ACD009AF8E49BF9C3E833F8E933F9306702612A
:100ADD005CE8FAE9FBD3E913FDE813FC885289536E
:100AED00C3EF94036038EF20E00DE82CF8E93DF9F1
:100AFD00ECFAEDFB020B17E828F8E939F9C3E82405
:100B0D0002F8E93400F97AFE7BFFC3EF9403400E3F
:100B1D008A548B55884E894F8C508D5161908854D5
:100B2D0089558A4E8B4F8C508D51306920C3E533DA
:100B3D0094034019E542A2E713F8E555F424013872
:100B4D00400B20E7087554FFF42401F5556190E83A
:100B5D00FAD3E813FC8852C3EF94036020EF20E032
:100B6D0007E82CF8ECFA617CE8282402F87AFEC339
:100B7D00EF940340088A54884E8C50619088548AB3
:100B8D004E8C50E56BC3335002646BF56B306002D5
:100B9D00619A753404D26043E680E52D5406601FDA
:100BAD00A840A941C2AF53E67F759100C3E498F503
:100BBD0094E499F595759104D26043E680D2AF2205
:100BCD00D265754400752000306B03752040020B13
:100BDD00ECD265754400752040306B03752000D252
:100BED00AF7801206722E52D54066002C265C3E58A
:100BFD00419405401378029405400878039405400C
:100C0D00027806306902780A206019E544601530D3
:100C1D00690AC3E53394034003D53406D2AFD26CD1
:100C2D0081CE71A2D2AF0000C2AF20672AE541C3C9
:100C3D00FB940F40027B0FEB240530730123306AC8
:100C4D0002742820620123F93069027982E58D133F
:100C5D00E58B13C39940B10544E59B5440B5200283
:0F0C6D0081B830690A08C3E8940A40010881156C
:100C7C0020650261ECC26553E67F75910030671008
:100C8C007594007595FC759104D26043E68061EC17
:100C9C00AE40AF41C3EE33FEEF33FF50047EFF7F17
:100CAC00FFC3E49EF594E49FF5958192C3E53394DC
:100CBC0002500261EC30650261ECD80281CC8115E6
:100CCC00C26C53E67F75910085549485559575914A
:100CDC0004854E56854F57D26043E680D2AFE52D42
:100CEC0054066008206A020533020D08306C0D2092
:100CFC006B0A206507158115810215B52278003025
:100D0C0064053065027801E53775F007A4F9E5F064
:100D1C0028F5F0E9A2F013A2F113A2F213F537C3F0
:100D2C0094785003753778C3E53795384008D26608
:100D3C00C292C294C296306002A14285505685512F
:100D4C0057D26043E68022D287207D11C2AF754313
:100D5C0002C295D293D2AF759F80020F2EC2AF758F
:100D6C004302C295D297D2AF759F80020F2EC287D5
:100D7C00307243207D20C2AF754303900175757EA0
:100D8C0020C296C297306204D294A19AD295D2AF67
:100D9C00759F89020F2EC2AF754303900175757E46
:100DAC0020C292C293306204D294A1BAD295D2AF2F
:100DBC00759F81020F2E207D17C2AF7543039001E2
:100DCC0050C296306202D294D2AF759F89020F2E18
:100DDC00C2AF754303900150C292306202D294D2DA
:100DEC00AF759F81020F2ED287207D11C2AF754344
:100DFC0004C293D297D2AF759F81020F2EC2AF75EA
:100E0C004304C297D293D2AF759F89020F2EC2872B
:100E1C00307243207D20C2AF754305900164757E0E
:100E2C0008C294C295306204D292C13AD293D2AF26
:100E3C00759F80020F2EC2AF754305900186757E9B
:100E4C0080C294C295306204D296C15AD297D2AF66
:100E5C00759F80020F2E207D17C2AF754305900140
:100E6C0046C294306202D292D2AF759F80020F2E8E
:100E7C00C2AF75430590015AC2943062EBD296D240
:100E8C00AF759F80020F2ED287207D11C2AF7543A4
:100E9C0006C297D295D2AF759F89020F2EC2AF753D
:100EAC004306C293D295D2AF759F81020F2EC28793
:100EBC00307242207D20C2AF754301900186757E51
:100ECC0080C292C293306204D296C1DAD297D2AF6A
:100EDC00759F81020F2EC2AF754301900164757E20
:100EEC0008C296C297306204D292C1FAD293D2AFA2
:100EFC00759F89E12E207D16C2AF75430190015A72
:100F0C00C292306202D296D2AF759F81E12EC2AFEF
:100F1C00754301900146C296306202D292D2AF75EF
:100F2C009F89C26622900144757E00C292C294C20F
:100F3C0096C293C295C297C26222788076FF0876D9
:100F4C00FF0876FF0876FF08760308760408760912
:100F5C00087603087601087601788C76010876FF0E
:100F6C000876FF0876FF0876FF0876FF08760308F8
:100F7C0076FF0876FF0876FF0876250876D0087687
:100F8C00FA0876FA0876040876FF087601087600E7
:100F9C0008767A0876FF087601087601087600084C
:100FAC007603227887E6FFC272BF0302D27278887A
:100FBC00E6C394036008C27DE630E102D27DC27EB6
:100FCC007889E630E102D27EC3EF94026008758E18
:100FDC0001D273020FE7758E00C273227880E6147B
:100FEC009000809378A4F67881E614900080937832
:100FFC00A5F67886E61490008D9378A6F6789CE694
:10100C007538FF75390CB402067538A075390AB4F9
:10101C00030675388275390578A3E61490009A9307
:10102C00F569120F3122C2A4C2A0789DE6B4010466
:10103C00D2A4C2A0B40204C2A4D2A0227896E6FA2A
:10104C007897E6FB7888E6B40305C3EB940EFB3087
:10105C007F047A007BFFC3EB9AFCC3948250027C22
:0E106C00827575000575EC8575F0A4C3E5F07E
:10107A00947D40F222D27F11481205FB7A007B0050
:10108A007C101205F1E55F2AFA74003BFBDCF37C65
:10109A0004C3EB13FBEA13FADCF7FEC27F11482202
:1010AA00E5EF20E6037520000520903FFFE52014B8
:1010BA006006901FFF1460009304600375EF1253DB
:1010CA00D9BF7581C043FF801205EC75EF0243B2A8
:1010DA0003E5B3240420E70DF521E5E320E00685C6
:1010EA0021B343E301120F317580FF75A48075F1B6
:1010FA00F075D4BF75900275A5FC75F2FD75D50221
:10110A0075A61175A0EE75F3F175E241E4F8F6D80B
:10111A00FD756B01120F46121600789886767530A7
:10112A0001C2AF1206051206151205FB12061C12A1
:10113A0005FB1206231205FB1217191206051206E1
:10114A0005120600C2AF78FA79FA308607D9FBD8B9
:10115A00F7021C00120FAF120FE8113211487898EB
:10116A008676120F3175B68075A900757D0075886F
:10117A005075891275C82475910475D84075A822CE
:10118A0075B80275E690759B80759D0075D10E75D0
:10119A00BC5875BB0975BA1175E8801205ECD2AF57
:1011AA001208A553DACF207E0343DA20307E0343A8
:1011BA00DA1043DA01C2D8C271120605D2617B0382
:1011CA007A0CE55E70077A0CDB0302114E1205FBFE
:1011DA0020700302114EC270E55FC3940240E1E53C
:1011EA002F541F856160F561B560D5DAD5C26153A8
:1011FA00DACF207E0343DA20307E0343DA10C2D8E6
:10120A00C27178A2E67008D274E52F54E0F52FC2B5
:10121A0075752900120600307409C3E529940A403D
:10122A0002D2751205F178023074027800C3E55FC4
:10123A009840F0C2AF120615120615120615D2AF63
:10124A00120605754D007888E6B40302612E120570
:10125A00F1788CE6C39401500302132EE530C3944F
:10126A0001500302132E207435C3E55F94FF500327
:10127A0002132EC2AF12062AD2AF120600C3E55FCE
:10128A00940150EFC2AF1206151205F6120615D2D6
:10129A00AF120600C3E55F94FF40E902179E7F057F
:1012AA00D27F1148120600C2AFC27F1148AE5FC397
:1012BA00E55F947FD2AF40761205ECC2AF12062AE0
:1012CA00D2AFDFDC117FC3EE94057897F6120605DC
:1012DA001216421217217F0AD27F1148120600C243
:1012EA00AFC27F1148AE5FC3E55F947FD2AF50E6CD
:1012FA001205ECC2AF1206151205F6120615D2AF88
:10130A00DFD6117FEE24057896F6120605121642EC
:10131A001217501206001148C3E55F94FF500241AC
:10132A007002179EC3E55F954D4003855F4D120617
:10133A000078017988E7B403027805C3E55F98402D
:10134A00024150C2AF12062A12062A12062AD2AF48
:10135A00120605753000E4F531F5320531E531F450
:10136A0070390532789AE678191460127832146066
:10137A000D787D14600878FA146003753200C3E5AD
:10138A003298401715327531B478998676C2AF1201
:10139A00062AD2AF789886761206001205F6E52A52
:1013AA007005307402214E78012074027806C3E574
:1013BA005F9840A77888E6C394036003120600E5A5
:1013CA002A700302114EC2AF120F31E4F522F5233F
:1013DA00F524F525F526F56AD2AF7885E6C333F507
:1013EA0068E4F545F546F547F548F549F573F52CF2
:1013FA00F52DF53775730875BB101205EC1208A99F
:10140A00E5E820ECFBA8BDA9BEE97001F8887412D2
:10141A0008AD75730875BB107887E6FE7602120F61
:10142A00AF7887EEF6C2AF7564FF1209258522648C
:10143A00852265852266D2AF75220175240175253C
:10144A000175260185636C756D0175B69075A903E2
:10145A00757D017888E6B40307C27D307602D27DB5
:0D146A00D268D269753300120E93120EBACB
:1014770012094512094C12094512094C1209450275
:101487001496C2AF120FAFD2AF75730075BB0912B6
:101497000BDE1206F5120D09120D5312094C120B31
:1014A700CD306D031206F620670312084830670334
:1014B70012088F120D09120D7A12094C120BDE3029
:1014C7006D03120732120D09120DF312094C120B9C
:1014D700CD306D03120790120D09120E1A12094C26
:1014E700120BDE306D031207ED120D09120E931267
:1014F700094C1208A9120BCD120D09120EBA1208C7
:10150700AD12094C306932206B2F8567648567659A
:1015170085636C756D0179187A0CC3E53399400CB6
:10152700C269D26A8A357564FF021540C3E55F94C4
:101537000140030214960215BD306A1B206B18E5A3
:1015470035147004C26A8189F535C3E55F9401409B
:10155700030214960215BD753600C3E562788298BA
:101567005054307404E52A604D7888E6B403172098
:101577007D05207607A18D307602A18D206B07D2DD
:101587006B85676481D578F0306B05856764782053
:10159700C3E5419850028196306B1BC26BC27D3008
:1015A7007602D27DD26A75351285676481960536D3
:1015B700E55F6002A1C0753600C2AF120F317887B0
:1015C700E6FE7602120FAF7887EEF6E4F522F523F2
:1015D700F524F525F526F568C26875B68075A90066
:1015E700757D00D2AF1205EC120F31307409C3E5D7
:1015F7003694054002214E6160901A0D782012162C
:1016070084E520B45A0CA3121684E520B4A503027E
:101617001622120F46121642021641901A037880BC
:101627007B0A121684A308DBF9901A0F788C7B18B3
:10163700121684A308DBF9901A2722C2AF1216C329
:1016470012169D901A00740E121689A374041216AE
:1016570089A37414121689901A0378807B0A1216CC
:1016670088A308DBF9901A0F788C7B18121688A3C9
:1016770008DBF91216D61216B4901A2722E493F64D
:1016870022E6438F01538FFD75EF0275B7A575B736
:10169700F1F0538FFE22438F02438F0175EF0275DE
:1016A700B7A575B7F1901A0DF0538FFC22901A0D5C
:1016B700745AD189901A0E74A5D189227A3079D0BB
:1016C7007820901A40D184E520F709A3DAF7227A27
:1016D7003079D0901A40E7D18909A3DAF922AB779C
:1016E700A878BB01027984BB02027985BB03027922
:1016F70086BB04027992BB05027987BB060279A3F0
:10170700BB0702799CBB08027988BB09027989E883
:10171700F7227C05120605DCFB22C2AF1206151262
:10172700061C12062312062A1205F61206151206C1
:101737001C12062312062A1205F612061512061C9B
:1017470012062312062AD2AF22C2AF12062A1206A7
:101757002312061C1206151205F612062A12062374
:1017670012061C1206151205F612062A1206231275
:10177700061C120615D2AF22AE77AF78C2AF12069B
:10178700151206151206151205F6DEF212062A12B2
:1017970005F6DFF8D2AF22F121F119F119757701BA
:1017A700757801757900F17F7C05AD5F120605C379
:1017B700ED955F70F5C3E55F9401400AC3E55F945B
:1017C700FF40320217DAD1E5D142F121C2AF75EFFE
:1017D70012F119DCD50579C3E5799403500280C667
:1017E700F1190578E5771490009F93F808C3E57819
:1017F70098500280AEF1191217190577C3E577944F
:101807000A5002809B120F46121642C2AF75EF12A2
:031817001217198C
:0319FD000210AA2B
:101A00000E0414FFFFFFFF0304090301015AA5019F
:101A1000FFFFFFFFFF03FFFFFF25D0FAFA04FF01DE
:081A2000007AFF01010003FF41
:101A400023506C6174696E756D3530417633232097
:101A500023424C48454C492346333930232020202B
:101A60002020202020202020202020202020202076
:101C0000C2AFC2D353D9BF7581C043B20343FF8073
:101C1000752438752503B1C975EF0275E24043F1AB
:101C20004053A4BF75D400D2867DFA780379E67C50
:101C300010752200752300901DD67B0675249875BB
:101C400025013086028142208608D8FBD9F9DCF7CD
:101C500081B4308608D8FBD9F9DCF781B4B189E4C6
:101C600093A3C39A6004DDC381B4DBDBB17B600264
:101C7000812B7B08E493FAA3B15CDBF87A30B15C8A
:101C8000752200752300B17BEAFCEBFDC3ED94FEE9
:101C9000400EB17B8A278B28ED30E0048A828B834B
:101CA000B17B7AC270D8C3ED94FE601350CEBD00F4
:101CB00025EC60097520007521FF0200008100A855
:101CC00027A9280809D804D90281D3B17FEA89AAB3
:101CD000F281C50D81A0C3ED94035049EDA2E092BD
:101CE000007AC5C3E5829400E583941C50902000DF
:101CF00010438F02438F0175B7A575B7F1F030001F
:101D00001FA827A9280809438F01538FFDD804D99C
:101D100002A12089AAE275B7A575B7F1F0A3A10DBC
:101D2000538FFC817C7AC1BD030CE493A3FAB140CC
:101D3000DCF8B138817C817EAA22AB23B15CEBFA5E
:101D4000EA6222752608C3E52313F523E52213F57D
:101D50002250066323A0632201D526EAB1C9B1C986
:101D600075260AEAF4200102D286300102C286B149
:101D7000C9C3134002C201D526EB22B17FEAFB2082
:101D80008602A17F308602A184752608AE24AF2585
:101D9000C3EF13FFEE13FEB1CDB1C9C3EA13308612
:101DA000024480FA30E703632201C3E52313F523DD
:101DB000E52213F52250066323A0632201D526D91C
:101DC000E52265236523F52222AE24AF250E0FDE22
:101DD000FEDFFCD20122424C48656C693437316326
:041DE000F390060175
:00000001FF
